:060000005522BE01E52BB4
:08000800542D820741345834E5
:100010003234353420345034493443342034643459
:10002000653463346F346434653472340034820769
:100030004734503453342F34573458342F344134E8
:100040005834203454347234203432342E34303422
:10005000003482074E346F34203453344D345434DA
:10006000203466346F3475346E3464342134003493
:100070008207203450344934433420343134363408
:100080004634363432347834203450346134633476
:100090006B346534743420344434653463346F34E1
:1000A00064346534723420342A3420344E3430348D
:1000B00051344234483420342834633429342034D1
:1000C00032343034303432342034263420344F3417
:1000D0004B343134563443344634203432343034A3
:1000E000303435340D340A34003403398207003497
:1000F0006434C8340F39820700340A3414341E348F
:10010000283432343C34463450345A340739820768
:1001100024344734503452344D3443342C3407396A
:1001200082072434473450344734473441342C3424
:1001300082070034063401340634013407340134B4
:1001400003340334043400340634003400340034FF
:1001500000340134023400340434013482070034A2
:100160000034063407340D340E3415341634193483
:100170001C34203400342034203420342034203403
:1001800021342334233427348400C501CC2884004F
:1001900000087520C500840A00087A20C507840A73
:1001A00000080F3945070800C6017F2105217F2976
:1001B000C4000A30450203180F29C508031D1E2973
:1001C000460886204406031D7F29C60A2C304406B3
:1001D000031D08005E30840030308000840A8000F7
:1001E000840A8000840A8000840A8000840A8000D7
:1001F000840A6B30840030308000840A8000840AD6
:100200008000840A8000BE136729483084003030A3
:100210008000840A0408703A031D072908000B3087
:10022000450203181E2946088F204406031D0800B6
:10023000C60A2C304406031D0800672944082C3ADE
:100240000319672945089820460603190800450840
:10025000073A031940294508083A03194029450877
:10026000133A0319402944082E3A03190800450897
:10027000AE204607483E840044088000C60A0800B5
:1002800044082E3A03195E294508AE20483E8400F2
:10029000840A000884038000840A840A0008840316
:1002A0008000840A4508133A031D5B29840A00086C
:1002B00084038000840A44088000080045089820D0
:1002C000C6000800AE20483E840000080800C601B1
:1002D000C50A4508153A031D080083210038031993
:1002E0007329061476290614E221DA239321F208F1
:1002F000031D7C29F8080319E221FD22BE13C60163
:10030000C5010610080002306221413A031D003485
:1003100010306221313A0319013410306221323A2F
:100320000319013400345E30C720C100C300C2018C
:10033000C10DC20DC10DC20DC10DC20DC10DC20D49
:100340004308C102031CC203F830C105C20CC10C32
:10035000C20CC10CC20CC10C5E308400B02108007C
:100360002F3080004108800AC10064304102031828
:10037000B3290008303A203003198000840A2F3056
:1003800080004108800AC1000A3041020318C229D6
:10039000840A4108303E800008000430F800F20171
:1003A000F001F10108002B30F7004430F20203188D
:1003B000DC29F2092D30F7007208C1007430840086
:1003C000B0210800F808031DE629CD21EB217108B2
:1003D000F200F80308002030F3003630F400031177
:1003E00000000519F00A0319F10AF30BF029F40BC8
:1003F000F1290800BA000000BA0BFC290800831696
:10040000A730810005168511831285110800BB00F5
:100410000A30BD0003108511031C85153930BE1844
:100420001A30FA210314BB0CBD0B0B2A08000D3047
:10043000202A08000A30202A08002030202A08003C
:10044000072A3B10051E00340930BD001330BE18CA
:100450000830FA210310051E0314BB0C3930BE18F6
:100460001A30FA210000BD0B2A2A3B08051A362A49
:100470003B14080021223B1C3A2A08007F398316CE
:100480009B001C141A08831208007F3983169B00F6
:100490008B131C1555309D00AA309D009C141C1117
:1004A0008B179C18512A8312080083160F30860080
:1004B00083120614612206103E1007303E22BF0050
:1004C0000800B7011E30B122303073222030732271
:1004D0002830A0220830A0220130A0220C30A02217
:1004E0000630A02208007A22061186108615A62260
:1004F00086110800B60037080F39F038B7008316A8
:100500008600831286100615861506088611861544
:1005100086118039031D822A061137080F39B7006A
:10052000831686008312360808007A220611861484
:100530008615A62286118615B60EA62286110800FB
:1005400073228615B60EA622861108000F30860586
:10055000F030360586040800A530B800B80BAE2A86
:100560000800B900AC22B90BB22A0800CD30A02295
:10057000BE189F23BE18BD2A98230800C030A022B1
:10058000F2080319DB2AD321533095224D309522EE
:10059000543095223A309522922377089522750897
:1005A000952276089522DF309522433095229223BA
:1005B000922392230800B40134082920003803193B
:1005C000E42A9522B40ADC2A08000130A022B401F2
:1005D0003408172000380319F02A9522B40AE82AB3
:1005E00008000130A022B4013408052000380319A6
:1005F000FC2A9522B40AF42A08000518052B3E1C93
:10060000032B3E10052B3E14052B8030A0228321A6
:10061000003803190D2B2A300319213095223F0889
:10062000343C0319152B3E18442B033062219522CC
:100630008E23DF3095228E238E2395238E238E23C7
:100640008E2392230730622195228E238E23A623A8
:10065000C030A0220530622195228E238E23DF3008
:1006600095228E238E2395238E238E238E239223F1
:100670001330622195228E238E238E238E233F08F2
:10068000343C0319442B08003F08343C031D4A2B1B
:100690009430A0220030622195228E233A30952298
:1006A0008E238E233A3095228E238E2392239223FB
:1006B0000730622195228E238E23A6233F08343CE7
:1006C000C0300319D430A022F2080319712BF808A6
:1006D0000319D3217508952276089522770895226B
:1006E000792B0230622195221030622195229223CB
:1006F000792B0930622195228E2395238E238E2318
:1007000095231130622195228E2392230830622195
:1007100095228E238E23DF3095220800840A00085C
:10072000952208002030952208002E3095220800DE
:10073000343095226B3095223830952208003930BC
:1007400095226B3095223630952208004B30952249
:100750006D30952208000130A022B0010800B00AD7
:100760003F08343C031DCD2B3008503C031C0800CF
:100770003008153A031DBF2BC030A022D72B3008FC
:10078000293A031DC62B9430A022D72B30083D3ABE
:10079000031DD72BD430A022D72B3008203C031CBC
:1007A00008003008113A031DD72BC030A0222808BA
:1007B000952208000614DF230610DF23080000003E
:1007C000B40BDF2BB50BDF2B08008B018312073036
:1007D0009F00FF21D42015266D27CD21E221E221A3
:1007E000E221E221DA23E522BE22851AFE2B051C36
:1007F000FC2B3E11BE10032CBE14032C0518022C3A
:100800003E15032C032CDA23B6226E2CBE1B162CAD
:10081000851E912C3E194D2C21223B1C062CB40028
:100820001B3A0319272C3408D820062C851A222CB1
:10083000051C1C2C0827262CBE13DA23DA23E522FC
:10084000B6226E2C0518262C0A27262C0C2C3A22B0
:10085000B4001B3A0319272C3408443A0319592CC5
:100860003408553A0319642C3408563A03196E2C8F
:100870003408523A03197A2C3408573A0319512F85
:100880003408773A0319342E34084D3A03194D2CA5
:100890003408723A0319832C062CBE13CD21E221B1
:1008A000E221E2210614E2210610BE22051C3E11BF
:1008B000062CB4013A2283169A008312340845228A
:1008C000B40AB41F5A2C062C80302022B4013408FC
:1008D0003E222022B40AB41F672C062CB40134082F
:1008E000172000380319772C2022B40A6F2C172206
:1008F0001A22062CB4013408840000082022B40A0D
:10090000031D7B2C062C8524062C4830840000080F
:100910002022840A0408703A031D872C17221A2209
:1009200008008316C130810083120530900000302A
:100930008B003E1350301026DA235525F122DA239E
:100940000610203084008001040A303C031CAA2CCD
:10095000840AA32CFF30AB00AC00A2308E00FB3029
:100960008F000C10051CE52B851E3E17AE25AA0C2A
:100970002A087E3A031DB22C0614AA010830A500ED
:10098000AE25031CCC2CA40AAA0C2408053A031992
:10099000CE2CA50BC02CE22CA401C42CAE25031830
:1009A000D32CA401C92CAE250318A02C2508033A8A
:1009B000031DA02CA401A91CBD2C23080F3C031867
:1009C000A02CF22CA91CA914A30A2308FF3A03198E
:1009D000A02C2308023C031C5F252E08AD002A082A
:1009E000AE00BD2C3E1BFF2CFF30AC06AB062D0825
:1009F0002C06031DA02C2E082B06031DA02C023054
:100A0000A302FF30A1000D30A700E425AF002F188E
:100A10000C2D0730A707052D2708A0000D3027064D
:100A200003191B2DAF1B192D0730A702E425AF00BA
:100A30000E2D2708A1000730A700AB23BE16752591
:100A40003E30A800D025AF23A701BE12752520088F
:100A50000D3A031D2E2D0D30A7003E2DBE122C3059
:100A6000A800D0250E30A7007525200827060319F9
:100A70003E2D2C30A800D025A70A342D3A30A800EE
:100A8000D0250230A707A202220803194D2DA70A7C
:100A9000E325A800D025AF23442D0D30A800D02594
:100AA0000A30A800D025A02C0900A0012008382079
:100AB000A800003A03190800D025A00A562DD22517
:100AC000A70A0830A500AD0C6825A50B632D08000A
:100AD00001300318AC060310AB0CAC0C031C08006F
:100AE0000830AC068430AB0608000630A600E325CB
:100AF000A8000310A80C2808203A031DD025BE1E0C
:100B0000852D2808203A031DAF23A70AA60B772DB1
:100B1000E325AF00AF0C0F30AF050319A42D2D3026
:100B2000A800D025BE1AAF230A302F02031C9E2D29
:100B3000AF003130A800D025BE1AAF232F08303EB9
:100B4000A800D025BE1AAF2321082706031DAD2D0E
:100B50002A30A800D025BE1AAF2308003E1AB32DB4
:100B6000B12DBE11B52DBE15B52D8518B82DBC2DD6
:100B70003E16BE1DC92DC02D3E12BE19C92DC02D59
:100B80000C1CAE2D16308E00FD308F000C1003149F
:100B90000800A2308E00FB308F000C1003100800FC
:100BA0002808202A220ABE3C031C0800A20AEE25BF
:100BB0002918DD2D2D08800008002D0883178000DE
:100BC000831329100800A203EE252918E92D000837
:100BD00008008317000883132910080027083E3CEB
:100BE0000318FD2D27088E3C0318012E2708BE3C54
:100BF0000318052EBE30A700052E2708413E8400AD
:100C000008002708613E840008006F302702840036
:100C1000291408003830A1000000A10B0C2E080098
:100C2000A0000A26A00B112E0800831602303E22D7
:100C3000FF0001303E22FE0003303E22FA00043065
:100C40003E22FB0005303E22FC0006303E22FD0025
:100C50003930A600A700A800AA00AB00AC002D30D8
:100C6000A5002030A9000800BE1706148316213005
:100C7000A0002008840083123A2283168417800083
:100C80008413A00A201F482EA01E482E201A4B2E87
:100C90007F06031D392E831250260C270610062CC2
:100CA00083162130A00020088400841700088413D4
:100CB0008312A00020087B060319762E20087C06EC
:100CC0000319DD2E20087D060319E82E8316A00ADD
:100CD000201F6E2EA01E6E2E201A742E8417000860
:100CE00084137F06031D532E83120800ED26A100F6
:100CF000ED26A200ED26A300ED26A4002108250282
:100D0000031CAD2E031DAC2E2118992E260822029D
:100D1000031CAD2E031DAC2E27082302031CAD2E91
:100D2000031DAC2E28082402031CAD2E031DAC2E7F
:100D3000AD2E22082602031CAD2E031DAC2E230867
:100D40002702031CAD2E031DAC2E24082802031C11
:100D5000AD2E031DAC2EAD2EF62629082102031C54
:100D6000DC2E031DDB2E2118C82E22082A02031CAC
:100D7000DC2E031DDB2E23082B02031CDC2E031D9F
:100D8000DB2E24082C02031CDC2E031DDB2EDC2EA4
:100D90002A082202031CDC2E031DDB2E2B08230253
:100DA000031CDC2E031DDB2E2C082402031CDC2E6E
:100DB000031DDB2EDC2EFF26662EED26AF00ED2672
:100DC000B000ED26B100ED26B200ED26B300662E90
:100DD000ED26AD00ED26AE00662E8316A00A200893
:100DE0008400841700088413831208002108A500DA
:100DF0002208A6002308A7002408A800080021084C
:100E0000A9002208AA002308AB002408AC000800AF
:100E1000F6260C2FFF260C2F8030A02221089522C9
:100E200022089522230895222E3095222408952207
:100E300043309522203095222F08952230089522A4
:100E400031089522320895222E30952233089522BA
:100E5000683095225030952261309522C030A02212
:100E60002D0895222E089522253095222030952296
:100E7000290895222A0895222B0895222E309522A2
:100E80002C08952243309522250895222608952284
:100E9000270895222E309522280895224330952246
:100EA000080083162130A000200884008417000861
:100EB0008413831220228316A00A201F632FA01EF2
:100EC000632F201A692F8417000884137F06031DDF
:100ED000542F831217221A22062C213084008417E3
:100EE00030308000840A8000840A8000840A2F3019
:100EF0008000840A30308000840A8000840A8000E8
:100F0000840A67308000840A30308000840A8000C0
:100F1000840A8000840A74308000840A30308000A3
:100F2000840A8000840A8000840A62308000840A77
:100F300030308000840A8000840A8000840A8000A7
:100F4000840A8000840A68308000840A303080007F
:100F5000840A8000840A0D308000840A20308000DA
:100F6000840A30308000840A8000840A8000840A69
:080F70004330800084130800E7
:02400E00020DA1
:1042000000002100430074000D00620068003200CD
:0E4210000000000000000000000000000000A0
:00000001FF
